:1000000000308A0004280000FF238316900000308F
:100010008A001E2827308400000803191D2801309B
:10002000A100A001A00B1228A10B11284A30A000AA
:10003000A00B18281B28800B0F28003484011F30C8
:1000400083050730990083160108C73908388100F5
:10005000831290010730990083160508033083123C
:10006000A000A00B312819088C1183169901851066
:10007000831285140630A600FA30A7000A20A60BCA
:100080003C2883168510831285100230A600FA30B2
:10009000A7000A20A60B4728831685108312851413
:1000A0000230A600FA30A7000A20A60B52288316B9
:1000B0008510831285100230A600FA30A7000A20AE
:1000C000A60B5D2883168510831285140230A600C6
:1000D000FA30A7000A20A60B682883168510831221
:1000E00085100230A600FA30A7000A20A60B73285C
:1000F00083160512831205160630A600FA30A700F3
:100100000A20A60B7E2883160512831205120230E0
:10011000A600FA30A7000A20A60B8928831605122C
:10012000831205160230A600FA30A7000A20A60B9B
:10013000942883160512831205120230A600FA30A5
:10014000A7000A20A60B9F28831605128312051606
:100150000230A600FA30A7000A20A60BAA288316B0
:100160000512831205120230A600FA30A7000A20F9
:10017000A60BB52883160512831205168316851063
:10018000831285140630A600FA30A7000A20A60BB9
:10019000C428831605128312051283168510831254
:1001A00085100630A600FA30A7000A20A60BD32837
:0601B000831637286300EE
:02400E009431EB
:00000001FF
